:1000000019C034C033C06EC431C030C02FC02EC040
:100010002DC02CC02BC08BC57FC628C027C026C0D2
:1000200025C0C8C693C692C691C693C695C69AC641
:10003000A5C6BAC611241FBE20E0A89521BD20E0A8
:1000400025BFE2E4FEE0A0E6B0E020E003C0C895F2
:1000500031960D92A236B207D1F7A2E6B0E020E0C9
:1000600001C01D92A63FB207E1F7ABC100C01895D1
:1000700088231CF0681730F404C060956F5F861702
:1000800008F4862F9927089587B9369A86B184FF98
:10009000FDCF0FB6F89484B10FBE95B1089587B91E
:1000A000369A86B184FFFDCF0FB6F89484B10FBEA7
:1000B00095B1969587959695879599270895282FB8
:1000C00030E0E0E0F0E845E050E8222314F46E2749
:1000D0007F27220F972F862F80709078892B41F0F1
:1000E000660F771F642775273F5F383070F303C0B2
:1000F000660F771FF9CF972F862F0895CF93DF9341
:10010000D091AE00DE5F1092800010927F00C0E0C0
:10011000CD1788F4EC2FFF27E355FF4F60917F0048
:10012000709180008081CBDF9093800080937F006E
:10013000CF5FCD1778F32DEA30E0F32FE22FEC0FED
:10014000F11D80917F0090918000892F99278083F5
:10015000CF5FF32FE22FEC0FF11D80917F008083A2
:10016000DF91CF910895CF93DF93D0919400DC5F1E
:1001700060E070E0C0E0CD1758F4EC2FFF27ED569B
:10018000FF4F80819CDF682F792FCF5FCD17A8F3B9
:10019000972F862FDF91CF910895982F963628F4C8
:1001A00086958695890F99270CC09A3940F09095CD
:1001B0009F5F892F86958695980F90959F5F892FD1
:1001C00099270895882341F0662319F0681718F4D9
:1001D000861B992703C0681B862F99270895CF9304
:1001E000DF93D82FC62FDC17F9F0DD23D9F06C2F61
:1001F0008D2FE8DF282F822F9927982F88270197A6
:10020000CD1770F42D2F222341F03327732F622F47
:10021000EFD5972F862F992709C08FEF90E006C062
:100220002C2FF1CFCC2319F780E090E0DF91CF9114
:10023000089582E034DF80937600843640F5F894A8
:1002400090E0969A9F5F9832E0F382E087B9369A01
:10025000AE9A90E0F8949F5F9630E0F3AE9896984F
:10026000789486B184FFFDCF0FB6F89484B10FBEA9
:1002700095B196958795969587958093F000909186
:100280007600981708F041C0891B8093F00082E047
:1002900006DF80937600843640F5F89482E087B9D3
:1002A00090E0959A9F5F9832E0F3369A90E0F89448
:1002B0009F5F9630E0F39598789486B184FFFDCFE8
:1002C0000FB6F89484B10FBE95B196958795969523
:1002D000879580936C00959880916C009091760042
:1002E000981780F4891B80936C0080917900882393
:1002F00079F090916C008091F00080936C00909365
:10030000F00006C010926C00F0CF1092F000BFCF4A
:10031000089590E0AA9AAC9AAB9A2091F000283008
:1003200020F480916C008830A0F060916C00822FE6
:1003300056DF893760F09091F00080916C0089174A
:1003400018F491E0AA9805C093E0AC9802C092E03E
:10035000AB98892F992787FD90950895813059F1A1
:1003600083B380FF03C083B381FF1BC09091620001
:1003700083B380FF0BC0923329F0992309F5909342
:1003800079001EC081E080937900F7CF83B381FFAD
:10039000F2CF992381F3892F815080936200982FA7
:1003A000EACF90916200923318F7892F8F5F809384
:1003B0006200982FDDCF1092620010927900D0CFAA
:1003C0000895CFE5D2E0DEBFCDBF82E083BF8FE9E5
:1003D00082BB8FEF81BB18BA8FE387BB1ABA1BBAF7
:1003E00085E886B98FE185BB8CEF84BB8BE085BD4A
:1003F0008CE083BD80E809B6082A09BE8FE289B97E
:10040000549A579A1092F5001092E60010927900D3
:100410001092CE0082E38093A70084E6809375005B
:1004200010926F0010926E001092ED001092EC008E
:10043000109284001092AA001092F40010928F0083
:1004400010926D00109277001092E80010926B00ED
:1004500081E084DFAE98949A1092E70078948091BE
:10046000840080FF7FC1979880916B008823B9F347
:10047000979A8CE00FB6F894A89581BD0FBE80E0E6
:100480006DDF80E00CDE8093EB0083E008DE80937C
:10049000EF0086E004DE8093780087E000DE809342
:1004A000AC008091AA00882309F45AC180916B00A6
:1004B000882309F453C18091AC00893408F44CC1FD
:1004C0009398C091D600C695C695C052D091D700DA
:1004D000D695D695D0528091E600C81B8091F50044
:1004E000D81B6FE18C2FC4DDC82F6FE18D2FC0DDCD
:1004F000D82F8C2F992787FD9095282F392F992356
:100500000CF425C1932F822F880F991F820F931F00
:1005100026E930E0281B390B8D2F992787FD909510
:10052000732F622F53D46AEF70E062D4972F862F17
:10053000D82F8C2F8D1B6FE19BDD8093F400CD0FA6
:100540006FE18C2F95DD80938F008091F4008E3FBA
:1005500008F4F8C01092F40090918F009E3F08F4C8
:10056000EBC010928F0090E0992331F099230CF4A6
:10057000E1C0935090938F008091F400882331F074
:1005800088230CF4D5C083508093F40080916B00D5
:10059000882309F4CAC08091DA0080936D008091AD
:1005A000DB00809377008091770083FF0EC08091FD
:1005B000D6008695869580528093E6008091D7007C
:1005C0008695869580528093F50010EEC0E209EF83
:1005D00027E090916D0093FF1DC0C093F400C0937D
:1005E0008F0085B382FF9EC085B384FF96C085B31C
:1005F00083FF8EC08091F4008D1B6FE139DD809305
:10060000F40080918F008D0F6FE132DD80938F00B9
:1006100090916D0096FF11C01093F400C0938F006D
:1006200085B382FF70C085B384FF68C085B3982FFF
:10063000987083FF5EC090916D0090FF0FC0C093D3
:10064000F40010938F0085B385B384FF4DC085B34C
:10065000982F987083FF43C090916D0095FF1BC049
:100660001093F40010938F0085B382FF35C085B3DB
:1006700084FF2DC085B383FF25C08091F4008D1BBE
:100680006FE1F6DC8093F40080918F008D0F6FE1B5
:10069000EFDC80938F0080917D00882371F039DE3C
:1006A000ACD090916D0091FD5FC080918D0081FF75
:1006B0005BC08BE48093750057C080E680937D001B
:1006C000B8DDEDCF1093F40010938F00D6CF1093C8
:1006D000F40000938F00CECF0093F400C8CF909326
:1006E000F40090938F00B8CF1093F400C0938F0064
:1006F000AECF9093F40090938F009DCF1093F400B1
:10070000C0938F0093CF10938F00C093F4008BCFD2
:10071000C093F400C0938F006DCF2093F400C0937A
:100720008F0065CF20938F005FCF80936D0039CF0E
:100730008D5F2ACF9D5F1ECF892F8150833008F0B7
:1007400013CF0FCF8150833008F006CF03CF22277D
:100750003327281B390BD6CE939AB3CE949AABCEBF
:1007600097D2A4CE979A80CE90938D0080917700F7
:100770008093EE0084CEFFCF982F992349F035EA7D
:1007800021E032BF28BF88B780FFFDCF9150C9F765
:100790000895CF93C82FCC2321F084E6EDDFC1501C
:1007A000E1F7CF9108958058681708F5982F961BA8
:1007B00096959695D1F020E02917E0F4681738F463
:1007C0004F5F5F4F4038510514F04FE750E08617F8
:1007D00040F4415050403FEF4038530714F440E894
:1007E0005FEF2F5F291750F305C091E0E4CF962FFC
:1007F000981BDECF952F842F08958091F400CDDCD7
:100800008093F40080918F00C8DC982F90938F0024
:1008100080917900882351F08091F40080958F5F5A
:1008200080938F0090959F5F9093F4009091F400D7
:10083000992309F447C084E18093F100992389F159
:1008400084E02DDC8093D20085E029DC8093820057
:1008500040916300509164006091D20080918F00BC
:10086000A2DF9093640080936300409165005091F3
:100870006600609182008091F40095DF282F392F67
:10088000309366002093650080916300909164002E
:1008900090939100809390003093720020937100A8
:1008A00017C080918F00882359F68091F10088232A
:1008B00039F6109264001092630010926600109254
:1008C000650006C080918F00882309F0B4CFB6CFB1
:1008D0000895992324F080958F77992702C08F7708
:1008E000907008951F920F920FB60F9211242F93BC
:1008F0003F934F935F936F937F938F939F93AF93A8
:10090000BF93EF93FF9380916800815080936800BC
:10091000882309F4DDC080917C00882309F4C8C0D5
:1009200080916A00882309F4B6C080917A0088BB60
:1009300010927A009091F200943058F480E1809304
:100940007A0080917400813009F4A3C082E1809321
:100950007A00892F81508093F2008F3F09F484C080
:1009600020916900243070F490917A00892F806280
:1009700080937A008091D000813009F473C098622E
:1009800090937A00822F8150809369008F3F09F401
:1009900054C0809178008A3110F010927A0041E0C2
:1009A000803108F040E02091F40030918F00822FD8
:1009B00083272CF480916D00817409F43CC0822F50
:1009C000992787FD9095992394F1429744F0832FBE
:1009D000992787FD9095992334F142970CF440E0D4
:1009E0004423F9F0809178008A30D8F4AE9A22231B
:1009F00079F08091E700813041F080916B0088238D
:100A000009F084C080937A0081C010927A00F5CFFB
:100A1000332379F78091F100882359F780937A0086
:100A2000E8CFAE98E4CF909581959F4FD6CF909523
:100A300081959F4FCACF482FC2CF8091710090916E
:100A4000720047DF8D5F8093690080917100909103
:100A50007200992324F081E08093D0009ACF109205
:100A6000D00097CF94628CCF8091900090919100AC
:100A700030DF8D5F8093F200809190009091910023
:100A8000992324F081E0809374006ACF109274005F
:100A900067CF81E15CCF8CE380936A008091EC00AA
:100AA0009091ED0001969093ED008093EC003DCF86
:100AB00084E680937C0080916A00882319F081503D
:100AC00080936A00809184008F5F8093840028CF98
:100AD00080EC8093680080917C00882319F081501D
:100AE00080937C0080916B00882329F080916B00BB
:100AF000815080936B008091F100882309F40BCF23
:100B00008091F10081508093F10005CFFF91EF912A
:100B1000BF91AF919F918F917F916F915F914F9115
:100B20003F912F910F900FBE0F901F9018951F921D
:100B30000F920FB60F921124EF92FF921F932F93F3
:100B40003F934F935F936F937F938F939F93AF9355
:100B5000BF93CF93DF93EF93FF931CB1809160001D
:100B600099278130910509F472C08230910584F48F
:100B7000892B09F071C0153509F06EC08091E9002C
:100B80009091EA00803F910509F066C081E062C063
:100B90008230910509F448C0039709F05DC0809147
:100BA0008C0063E9E62E60E0F62EFF2DEE2DE80FB7
:100BB000F11D10838F5F80938C00C0916700C1503E
:100BC000C0936700CC2309F047C0CDDAF92FE82F96
:100BD0003097D1F5809193008130B1F54C2F809101
:100BE0009400282F33272E5F3F4FE217F307B4F40A
:100BF000AE2FBF2FC3EDD0E07F2D6E2DFB2FEA2F40
:100C0000EC0FFD1FA60FB71F8C9180834F5F842FC1
:100C10009927B92FA82FA217B30784F3949885E0DA
:100C200080936B00A89510C01093940083E080938C
:100C3000600082E080938C00812F8E5F809367003C
:100C400099270496459744F01092600005C01093D0
:100C5000930082E080936000812F99279093EA00AF
:100C60008093E900FF91EF91DF91CF91BF91AF9118
:100C70009F918F917F916F915F914F913F912F91B4
:100C80001F91FF90EF900F900FBE0F901F9018953F
:100C90001F9381E08093AD0012E08093AF008091BC
:100CA000F4008093B00080918F008093B100809118
:100CB00078008093B2008091EF008093B300809120
:100CC000AC008093B40080918A008093B50080913D
:100CD000AB008093B60080916D008093B700809147
:100CE00077008093B800809184008093B900912FA1
:100CF000955F809182008093BA008091D2008093AA
:100D0000BB009093AE00FAD91093AA00539A559A5B
:100D10008FEF8CB91F9108951F920F920FB60F920B
:100D200011242F938F939F93AF93BF93EF93FF93D0
:100D30002091AA00822F9927AA27BB27F92FE82FF5
:100D4000E930F105B8F5EF5EFF4F09948FEF8CB9EC
:100D500005C080EF8CB902C085E58CB92F5F209368
:100D6000AA0028C0109273008091AE008C5F80931F
:100D7000E5008091AA008F5F8093AA009091730094
:100D8000EDEAF0E0E90FF11D80818CB99F5F90934F
:100D900073008091E50081508093E500882351F431
:100DA00088E08093AA0006C01092AA008FEF8CB949
:100DB00055985398FF91EF91BF91AF919F918F916B
:100DC0002F910F900FBE0F901F901895552700245C
:100DD00080FF02C0060E571F660F771F6115710551
:100DE00021F096958795009799F7952F802D089576
:100DF00097FB092E07260AD077FD04D00CD006D029
:100E000000201AF4709561957F4F0895F6F790953C
:100E100081959F4F0895AA1BBB1B51E107C0AA1FD4
:100E2000BB1FA617B70710F0A61BB70B881F991F8B
:100E30005A95A9F780959095682F792F8A2F9B2F27
:020E4000089513
:020E42000000AE
:00000001FF
